:100000001529A501A400B7172730A300103014202C
:100010000330A300E8301420A30164301420A301AE
:100020000A30142024081F28A2002508A100240853
:10003000A000F4202008031DB713B71B0800303EB2
:10004000A6003A0884000930A70003102C20A60C53
:10005000A70B262803142C288413B71D3B2800085F
:100060003804371D38068000841700083804031C44
:1000700038068000462800083804031C3806371963
:10008000380680008417380980054628370D063960
:10009000A0004F20A100A00A4F200000BC28003083
:1000A0008A002008820701348B3403342B34003457
:1000B00052340C34EF34A3003A08840038098B2002
:1000C0008413A30803191029F030A50022088038F2
:1000D000A400F030A5030319A5000319A303031915
:1000E00010292008A6002108A7001630BB202608EA
:1000F000A0002708A1009F20030120183808A21F94
:100100003808A20803190301A40F8828800666286E
:10011000892800006928841780051029A000A00DF7
:10012000A00D200D383941389F000030A100323039
:10013000BC201F151F199A28A1011E08102921088B
:1001400020040319A00A8030201AA1062019A10654
:10015000A018A106210DA00DA10D1029A301A20038
:10016000FF30A207031CA307031C10290330A100C2
:10017000E330BC20B028A101F43EA000A109FE306C
:10018000031CC528A0070318C228A0076400A10FFC
:10019000C22800002018CC282018CE280800A10171
:1001A000A301A2000130D928A101A301A2000430BB
:1001B000D928A80023082102031DE02822082002D4
:1001C000043003180130031902302805031DFF30E5
:1001D00010290038031DFF300405031DFF301029CE
:1001E0000404031DFF301029A501A4011030A6004E
:1001F000210DA40DA50D2208A4022308031C230F22
:10020000A50203180A292208A40723080318230FAC
:10021000A5070310A00DA10DA60BF8282008102992
:100220008313031383126400080083161F308500B4
:10023000860170308F008312061083160610831219
:1002400086108316861083120611831606118312F8
:1002500086118316861183120612831606128312E4
:1002600086128316861283120613831606138312D0
:100270008030BE007730BF000130C10083169F017F
:1002800006308312BA004030B8006430A2000A3051
:100290005B205A30A20005305B205030A2000530B0
:1002A0005B206E30A2000A305B200630BA0040307E
:1002B000B8006430A20005305B206E30A20005302B
:1002C0005B20061283160612831286168316861288
:1002D000831260220630BA004030B8005030A200CD
:1002E00005305B205A30A20005305B208612831651
:1002F000861283120616831606128312A022063077
:10030000BA004030B8006430A20005305B206E3087
:10031000A20005305B200612831606128312861691
:10032000831686128312E0210630BA004030B800EE
:100330005030A20005305B205A30A20005305B200F
:1003400086128316861283120616831606128312ED
:10035000202202308E20BC003C08A0006430CF2058
:10036000B2003C08A0008230D420B40032088400DF
:100370003408E920B400B5006400340835040319DA
:10038000DD290630BA004030B8006430A2000A30DF
:100390005B205A30A20005305B206430A20005309B
:1003A0005B206E30A2000A305B205030A200143077
:1003B0005B205A30A20014305B20A9296300DE299B
:1003C000C00106108316061083128610831686104D
:1003D000831286148316861083120130A300903096
:1003E000AF2041083E02B200B301031CB303400832
:1003F000A000A1013308A3003208D620B2003E08B5
:100400004107B400B501B50D4008A000A1013508B1
:10041000A3003408D120B400320884003408F0204E
:10042000B400B50064003408350403191B2A0130F8
:100430008E20C000F12986108316861083120800D2
:10044000C0010610831606108312861083168610CC
:10045000831206148316061083120130A3002C3079
:10046000AF2041083F02B200B301031CB3034008B0
:10047000A000A1013308A3003208D620B2003F0833
:100480004107B400B501B50D4008A000A101350831
:10049000A3003408D120B400320884003408F020CE
:1004A000B400B50064003408350403195B2A013038
:1004B0008E20C000312A0610831606108312080011
:1004C000BD0106118316061183128611831686114B
:1004D000831206158316061183120130A300903093
:1004E000AF2041083E02B200B301031CB3033D0834
:1004F000A000A1013308A3003208D620B2003E08B4
:100500004107B400B501B50D3D08A000A1013508B3
:10051000A3003408D120B400320884003408F0204D
:10052000B400B50064003408350403199B2A003078
:100530008E20BD00712A0611831606118312080051
:10054000BD010611831606118312861183168611CA
:10055000831286158316861183120130A3002C3076
:10056000AF2041083F02B200B301031CB3033D08B2
:10057000A000A1013308A3003208D620B2003F0832
:100580004107B400B501B50D3D08A000A101350833
:10059000A3003408D120B400320884003408F020CD
:1005A000B400B5006400340835040319DB2A0030B8
:1005B0008E20BD00B12A8611831686118312080091
:1005C00000308E20BD000630BA008030B800043004
:1005D000B700FE302020803020204C3020203A30E0
:1005E00020203D0801202030202020302020013014
:1005F0008E20C0000630BA008030B8000430B7004A
:10060000FE30202086302020523020203A3020201A
:1006100040080120203020202030202002308E2071
:10062000BC000630BA008030B8000430B700FE309D
:100630002020C030202049302020523020203A3065
:1006400020203C08012020302020203020200800DD
:02400E00303F41
:00000001FF
